:105F810001130000090101240200000301FA0400C9
:105F9100FA0500030A0A5A0B001E0C00FA0D000351
:105FA1000E00030F0164100096120132130AFA1455
:105FB100010215000217010A1801FA1905321A0126
:105FC1000A1B01FA1C05321FFFFF20FFFF23011EE0
:105FD1002400642A00FA2B00FA2C50782D003D2E63
:105FE10000462F001E3000643250783432FA3501F9
:105FF10064360164370150380A643C00643E003C59
:106001003F000140FFFF411450420A5A430AC8446D
:1060110005324500B44600FA4701484802034C00E6
:10602100FA4EFFFF500404510596520A32530B46B3
:10603100540A96560102570546580002590A465A13
:1060410032FA5B010A5C0A325E000A5F00FE61FF00
:10605100FF6402106600026701016A0A3C6B0000DE
:106061006C32967300007400007801327901327E3F
:10607100FFFF81FFFF84FFFF8500AF8600018700DE
:10608100FA89010A8A00009900009D0A969E000182
:106091009FFFFFFAFAFA0065006F00790083008D17
:1060A100009700A100AC00B600C000CA00D400DE19
:1060B10000E800F2005B0063006A0072007A00826F
:1060C10000890091009900A100A800B000B800BFAC
:1060D10000C700CF00D600DF00E600EE00F600406A
:1060E1000046004C00520059005F0065006B0071D2
:1060F1000077007D00830089008F0095009C00A23D
:1061010000A800AE00B400BA00C000C600CC00D2A6
:0A61110000D900DF00E500EB00F10B
:1035E7009007BAE0FEA3E0FF905F83126254E49372
:1035F700F599905F81E493FC740193FDEFB505079E
:10360700EEB50403754D009007BA12623B2285F9A7
:103617007285FA737E017F00E57312622DE5722FC2
:10362700FF50010E8E598F5A900013E0FCA3E0FD66
:10363700EF2DFDEE3CFC8C5B8D5C2275A71085F9A8
:103647007285FA737E017F00E57312622DE5722F92
:10365700FF50010E8E598F5A9000DCE0B40210AC77
:103667002CAD2DEF2DFDEE3CFC8C5B8D5C8016AEFA
:1036770059AF5A900013E0FCA3E0FDEF2DFDEE3C9F
:10368700FC8C5B8D5C22AE59AF5A740A8E048F0591
:10369700FF12621D8C5B8D5CAE59AF5A740A8E04A3
:1036A7008F05FF1262488C598D5AE55A45596013A8
:1036B700740AC3955AFFE49559FE8E598F5A785B61
:1036C700126281E572A85BB80015D3955C4010E5DE
:1036D70072C3955CFFE4955BFE8E5B8F5C8010E5A3
:1036E700722424C3955CFFE4955BFE8E5B8F5C754B
:1036F7007200AE5BAF5C74116F4E600674126F4E52
:103707007018AE5BAF5C74116F4E700575720180F7
:1037170003757202755C10755B00AE5BAF5C741469
:103727006F4E600674156F4E7018AE5BAF5C741405
:103737006F4E70057572018003757202755C1375A3
:103747005B00AE5BAF5C74236F4E600674246F4EF4
:103757007018AE5BAF5C74236F4E70057572018095
:1037670003757202755C22755B002290008AE0B4D3
:103777000104C2108002D21090008BE0B40104C291
:10378700118002D2119000C8E075F0DCA4FFAEF002
:10379700740A8E048F05FF12621D9007B0ECF0A328
:1037A700EDF0A20D401674038C068D0712622D747E
:1037B700011200399007AEEEF0A3EFF07E017F0013
:1037C700900086E012622D9000C9E08E048F05FFFD
:1037D70012621D740AFF12621D8D5F9000D2E075A0
:1037E700F0DCA4FFAEF0740A8E048F05FF12621D91
:1037F7009007B4ECF0A3EDF09000D4E060139000D4
:10380700D4E0F5F0741684FF7E00EF9007BEF080D9
:103817000674649007BEF09000CAE090006EF090C6
:103827000114E0900058F09000A3E090005AF09047
:1038370000CCE090005BF0900078E090005CF090A6
:1038470000FEE0900061F074E390006DF09000B32B
:10385700E0B40B0874E390006DF0805A9000B3E079
:10386700B419129000C9E090608212008CE4939022
:10387700006DF080419000B3E0B41E129000C9E0E3
:103887009060A012008CE49390006DF08028900067
:10389700B3E0B428129000C9E09060CA12008CE42B
:1038A7009390006DF0800F9000B3E0B4460890004D
:1038B700AAE090006DF0900071E0FE9000B0E0B5D6
:1038C7000633900073E0FE9000CEE0B50627900027
:1038D70072E0FE9000DCE0B5061B900075E0FE90FC
:1038E7000083E0B5060F900074E0FE9000BEE06E26
:1038F7007003023A3C900049E0C3940550087402F3
:103907009000FFF080149000DCE0600874089000DD
:10391700FFF08006740A9000FFF0900083E0B40186
:103927000674009000E9F0900083E0B4020674008A
:103937009000CEF0900083E0B4030674009000DBA3
:10394700F09000CEE0D3940140147418900101F078
:1039570074009006C8F074009006C9F0800C7400DB
:10396700900101F074189006C8F09000B0E0601460
:10397700741A900097F074009006D0F074009006C7
:10398700D1F0800C7400900097F0741A9006D0F074
:103997009000B0E0B402147419900098F07400908D
:1039A70006CCF074009006CDF0800C74009000985F
:1039B700F074199006CCF09000DCE0700E7405905E
:1039C70006DCF074069006E0F0801874009006DCC0
:1039D700F074009006DDF074009006E0F07400903B
:1039E70006E1F0D2269000B0E0900071F09000DC84
:1039F700E0900072F09000CEE0900073F09000BE6F
:103A0700E0900074F0900083E0900075F0900083E0
:103A1700E0900059F09000BEE090005DF09000DC6F
:103A2700E090005EF09000B0E090005FF09000CE74
:103A3700E0900060F09000E6E0B4011790001F747A
:103A47000FF0A374FFF0900021E4F0A3F07402904C
:103A570000E6F09000E6E0B40341900021E0FEA309
:103A6700E0FF90001FE0FCA3E0FD126279741012E2
:103A7700622D7408120039EF90006AF0EF70067437
:103A8700FF90006AF074009000E6F0900020E0904C
:103A9700006BF090001FE090006CF0900077E090D2
:103AA700003BF090003BE0241290003CF090003C7B
:103AB700E0D39424400B90003CE0C3942490003C56
:103AC700F090003FE4F090003BE064116007900045
:103AD7003BE0B4122090003BE0B411067402900062
:103AE7003FF090003BE0B4120690003F7401F07481
:103AF7001390003BF090003BE06414600790003B9C
:103B0700E0B4152090003BE0B41406740290003F27
:103B1700F090003BE0B4150690003F7401F0741676
:103B270090003BF090003BE06423600790003BE08F
:103B3700B4242090003BE0B42306740290003FF0C9
:103B470090003BE0B4240690003F7401F090003BE6
:103B57007401F0900040E4F090003CE064116007CD
:103B670090003CE0B4122090003CE0B411067402CF
:103B7700900040F090003CE0B412069000407401C1
:103B8700F0741390003CF090003CE06414600790E0
:103B9700003CE0B4152090003CE0B4140674029099
:103BA7000040F090003CE0B415069000407401F02E
:103BB700741690003CF090003CE06423600790008E
:103BC7003CE0B4242090003CE0B42306740290004B
:103BD70040F090003CE0B424069000407401F0905F
:103BE700003C7401F0900077E0FE9000DAE02E9040
:103BF7000042F0900042E064036017900042E064E6
:103C070012600F900042E064156007900042E0B434
:103C17002406900042E004F0900042E0640260173E
:103C2700900042E06411600F900042E06414600766
:103C3700900042E0B42306900042E014F090004266
:103C4700E0D39424400B900042E0C39424900042B8
:103C5700F0900042E0D39412400D900042E0C394EC
:103C670012900043F0800A900042E0241290004333
:103C7700F07550129000BDE090003DF090003DE0DF
:103C8700B4020690003D7401F090003DE0B40306D5
:103C9700740490003DF090003DE0B411067410905C
:103CA700003DF090003DE0B41206741390003DF023
:103CB70090003DE0B41406741390003DF090003D71
:103CC700E0B41506741690003DF090003DE0B42373
:103CD70006742290003DF090003DE0B42406742560
:103CE70090003DF090003DE0B42606742590003D1D
:103CF700F090003DE0B42706742890003DF0900056
:103D07003DE0B43506743490003DF090003DE0B4DA
:103D17003606743790003DF090003DE0B4380674E5
:103D27003790003DF090003DE0B43906743A9000BA
:103D37003DF090003DE0B44706744690003DF0909A
:103D4700003DE0B4480690003D7401F090003DE06E
:103D5700D39424400F90003DE0C3942490003DF09D
:103D6700D2208002C22090003DE0D39412400D90F3
:103D7700003DE0C3941290003EF0800A90003DE0C1
:103D8700241290003EF022C293C294C291C292C202
:103D970087C290E5B554EFF5B5E5B554DFF5B5C283
:103DA70096C295C2A0C297C2A2C2A1E5B554BFF5FB
:103DB700B5E5B5547FF5B5E5B554FBF5B5C2127554
:103DC7005D469000C0E07005756C028003756C035A
:103DD70075540075530090000874FFF0A374DCF06D
:103DE700C217C21974C8900033F074C8900037F036
:103DF700755200755100C20D754600E56EB4090392
:103E0700756E00756200900015E4F0A3F0756F10F1
:103E1700C215C2169007B0E0FEA3E0FF740312625A
:103E27002D74011200399007AEEEF0A3EFF0C20235
:103E370075560075550090000CE4F0A3F0C2277585
:103E47005800755700900082E075F032A4FDACF081
:103E570090001DECF0A3EDF0C2372285F97285FAC8
:103E6700737E017F00E57312622DE5722FFF50010B
:103E77000E8E598F5AAC5BAD5CEF2DFDEE3CFC8C82
:103E87005B8D5CD293D294E55CF5FBE55BF5FCE5D5
:103E97005CF5E9E55BF5EA9000BEE0B40314D29166
:103EA700D292E55CF5EBE55BF5ECE55CF5EDE55B02
:103EB700F5EE2275A71085F97285FA737E017F00EA
:103EC700E57312622DE5722FFF50010E8E598F5A3E
:103ED7007E017F769000FBE012622DAC59AD5AED62
:103EE7002FFFEC3EFE8E5B8F5CE55CF5FDE55BF539
:103EF700FE90006EE4F075A7007412900045F02262
:103F070085F97285FA737E017F00E57312622DE5EC
:103F1700722FFF50010E8E598F5A9007B0E0FCA305
:103F2700E0FDEF2DFDEE3CFC8C5B8D5CE55CF5FD6B
:103F3700E55BF5FE220563229000BEE0B4035390D3
:103F470000DCE0B4012EA2D8B34004C293C287A21A
:103F5700D9B34004C294C290A2DAB34008C291E533
:103F6700B554EFF5B5A2DBB34008C292E5B554DF0F
:103F7700F5B5801CA2D8B34002C293A2D9B34002C0
:103F8700C294A2DAB34002C291A2DBB34002C2924A
:103F9700801EA2D8B3400AC2939000DCE06002C240
:103FA70087A2D9B3400AC2949000DCE06002C290B5
:103FB700A2DCB34004C296C29575D8402285A7718A
:103FC70075A710A2D8B34002C287A2D9B34002C2D4
:103FD70090A2DAB34006E5B554EFF5B5A2DBB340DE
:103FE70006E5B554DFF5B5A2DCB340089000CAE09A
:103FF70090006EF075D8408571A722900047E49332
:104007006406600280FE74C89007B6F8E4F0E8A37F
:10401700F075B50075840175A70075FFA090004184
:10402700E4F075C91075A70F75A1C775A70075D9F5
:104037000075CE0C75A70F75F1FE75F2FF75F307C6
:1040470075F47875A4BA75A5FF75A60775AE0075E2
:10405700AFFF75D48175D5FF75D6FF75D7FF75A7E7
:104067000075A20175A14775F80975D80075D904BF
:1040770075DA0975DB0975DC0975DD0975DE097502
:10408700D84075A71075D80075D90475DA0975DB9E
:104097000975DC0975DD0975DE0975D84075A70056
:1040A70075E60875E71075BC0175BE0475BD6C75BE
:1040B700BE0775BDA075BE0875BD0175BC0075BB93
:1040C7001875BC2075BA0875E88075D11375A70FE8
:1040D70075E10575E20075C740123D8E759700754D
:1040E7009780740A12620D7597C0E5975420700285
:1040F70080F8758F0275A700D2AF75980075A90C67
:1041070075A70F75AB4375ADFB75AC1E75A710751D
:10411700C91875CA0075CB0075C80475A7007589DD
:1041270012758E04758C00758A00C2A9D28C758DA4
:1041370000758B00D2ABD28E75EF0675D944C29944
:1041470074C8F5097508001200E375B5001204E399
:1041570074639007B6F8E4F0E8A3F012036F74C82D
:104167009007B6F8E4F0E8A3F07464F50975080061
:104177001200E3900059E0900083F0C21D90008385
:10418700E0D3940340067400900083F0900083E02E
:10419700905B99F82828738028A2B44002D21D802A
:1041A7002075A70F75F30F75A700A2A34002D21DB4
:1041B700800F75A70F75F31775A700A2A44002D249
:0141C7001DDA
:0C5B990002419E0241A00241A80241B955
:1041C800A21DB34066757208E572D3940E5020E5BF
:1041D800729007B6F8E4F0E8A3F012023E7464F5B2
:1041E800097508001200E37872740126F650D97434
:1041F800029000BFF0900083E0D39403400674005F
:10420800900083F0900083E0905BA5F828287380E5
:104218001674009000E9F0800E74009000CEF080D3
:074228000674009000DBF0BA
:0C5BA5000242170242190242210242296A
:10422F00D21C8064757201E572D394075020E57239
:10423F009007B6F8E4F0E8A3F012023E7464F509B3
:10424F007508001200E37872740126F650D97401D4
:10425F009000BFF0900083E0D39403400674009069
:10426F000083F0900083E0905BB1F82828738016EC
:10427F0074009000E9F0800E74009000CEF080067C
:06428F0074009000DBF05A
:0C5BB10002427D02427F02428702428FC6
:10429500C21C900058E0900114F0900059E0900085
:1042A50083F090005AE09000A3F090005BE090004E
:1042B500CCF090005CE0900078F090005DE090001C
:1042C500BEF090005EE09000DCF090005FE09000B2
:1042D500B0F0900060E09000CEF0900061E09000BA
:1042E500FEF09000C9E07006740A9000C9F09000D5
:1042F500AAE0700674E39000AAF09000B0E0049084
:104305000071F0123772E5B54401F5B574069000F9
:1043150047F07401900048F0740390004AF074056A
:1043250090004BF0742D90004CF0740590004DF00A
:10433500740090004EF07400900053F074009000EB
:1043450054F07401900055F07400900056F074FF1D
:10435500900057F0745390014DF0747590014EF034
:10436500746290014FF07461900150F07472900185
:1043750051F07475900152F07420900153F074342B
:10438500900154F07443900155F07479900156F002
:10439500746C900157F07420900158F074339001BB
:1043A50059F0743690015AF0745490015BF0900006
:1043B500E5E090006AF090009CE090006BF09000C2
:1043C5009DE090006CF0A2B6B3920EA2B3B3920F2B
:1043D500A2A4B39223A2B4B39224A2A3B39225902C
:1043E5000066E4F0756E00743A900776F074FD90FF
:1043F5000777F0900067E4F09007B0E0FEA3E0FFD8
:10440500740312622D74011200399007AEEEF0A309
:10441500EFF0756D01900045E4F0C222756200C2AF
:1044250013D214C202757000C229D203C22AD20463
:10443500C22BD205C22CD206C22DD207C22ED2085B
:10444500C22FD209C230D20AC231D20BC232D20C2B
:10445500C21EC21FC220C221C22612009E755E0066
:10446500756A00756000756432756500756600755E
:104475006700756800756900900015E4F0A3F07594
:104485006B00D2B2D2A4D2B0D2B1D2A3D2A7D2A657
:10449500D2A5D2B7900082E0D394FA400674FA9080
:1044A5000082F07E017F0090006CE012622D90008A
:1044B5006BE02FFF50010E90001FEEF0A3EFF0EF21
:1044C500D394FFEE940F400790001FE4F0A3F09003
:1044D500006AE0700674FF90006AF074009000A90D
:1044E500F09000BFE0D39402400674019000BFF045
:1044F5009000C0E07005756C028003756C03900038
:10450500C1E0D39401400674009000C1F09000C74B
:10451500E0C3940A5006740A9000C7F09000D1E0F9
:10452500700674019000D1F09000D1E0B4FF0674DC
:10453500FE9000D1F09000D8E0D394FE400674FEC2
:104545009000D8F09000FEE0D394024006740190EC
:1045550000FEF0900114E0D394014006740190012F
:1045650014F074019000DEF074019000DFF0740027
:104575009000E6F07400900102F07400900106F0DE
:1045850074299006BCF0742A9006C0F07417900642
:10459500C4F0741B9006D4F0741C9006D8F0D29C1D
:1045A5009000B1E0D39404400674049000B1F090FB
:1045B50000E3E0D39404400674049000E3F0E56F53
:1045C500D394104003756F109006BDE0D3940C4052
:1045D5000674009006BDF09006C1E0D3940C400629
:1045E50074009006C1F09006C5E0D3940C400674A3
:1045F500009006C5F09006C9E0D3940C40067400FF
:104605009006C9F09006CDE0D3940C400674009056
:1046150006CDF09006D1E0D3940C400674009006C8
:10462500D1F09006D5E0D3940C400674009006D5E1
:10463500F09006D9E0D3940C400674009006D9F0AA
:104645009006DDE0D3940C400674009006DDF090F2
:1046550006E1E0D3940C400674009006E1F0D2EC3C
:1046650075CF01A298B34005C298120616E54D60B4
:1046750006A299B3B340028005C299120AB4E54E69
:1046850064016005E54EB4040280D5C28E7E107FBC
:1046950000E56312622DE58D75F010A4FDACF0EF19
:1046A5002DFDEE3CFCE58B75F01084FF7E00ED2FB3
:1046B500FFEC3EFE8E538F54D28E9000A3E060092E
:1046C5009000A3E0C3943D4002805C900017126205
:1046D5003B900017E0FEA3E0FF900019E0FCA3E08B
:1046E500FDEFB50542EEB5043EB21BA20DB3401970
:1046F50075E700A21BB34008E5B54404F5B580068F
:10470500E5B554FBF5B575E710900019E0FEA3E09B
:10471500FF90001BE0FCA3E0FDEF2DFDEE3CFC90BF
:104725000019ECF0A3EDF09000B0E060099000B046
:10473500E0C394034002806F1229C0A20DB3500953
:10474500900066E0C3942B4002800690009AE0F545
:1047550045E54575F005A4FFAEF09007B8EEF0A36A
:10476500EFF0900087E0C395604007E55EC3955F75
:1047750050079007B8E4F0A3F0AE2EAF2F9007B81E
:10478500E0FCA3E0FDEFD39DEE9C4004C2A1800BAD
:10479500900066E0C394415002D2A19000B0E0B40D
:1047A5000205A2A1B392A29000B0E0B4031C122AA4
:1047B500DBAE2EAF2F9007B8E0FCA3E0FDEFD39D55
:1047C500EE9C4004D2A18002C2A190008BE060095A
:1047D500A2B3300F01B3B340028039A2B3300F0149
:1047E500B34031A2B3301101B3401C9000BEE0B418
:1047F5000306A21EB3B3400280067404900045F080
:10480500D21EA211B3920FA211B330B301B340046B
:10481500A211920FA2B6300E01B35003024EA8A208
:10482500B6300E01B35003024EA8A2B6301001B344
:104835005003024CCD756D009000A3E0B43D197591
:10484500E700A210B34008E5B554FBF5B58006E5D1
:10485500B54404F5B575E710055DA212B3B3501361
:10486500AE53AF54900008E0FCA3E0FDEDC39FEC10
:104875009E40030249CFE55DB41106755D130249FB
:10488500B2E56CB4032EA227B34022E55DB4230341
:10489500756C01E55DC3942350069000457401F0E5
:1048A500E55DD3942340067402900045F0755D01E3
:1048B500D227805AE56CB40206756C01755D23E557
:1048C5005DB42305755D018045900045E07030E5D8
:1048D5005DC3942350069000457401F0E55DD394C3
:1048E5002340067402900045F0E55DC39423500211
:1048F500D222E55DD394234002D222C296C295907E
:1049050000C0E0B40105123D8E8003755D01900085
:10491500A3E060099000A3E0C3943D40028043906A
:104925000017E0FEA3E0FF9000A3E08E048F05FFD3
:1049350012621D74018C068D0712003990001BEE62
:10494500F0A3EFF090001BE0F8A3E0900019C8F089
:10495500A3C8F0900017E4F0A3F0C21BE5B554FB23
:10496500F5B5A2B4B34002C224A2A4B34002C22347
:10497500A2A3B34002C225A222B34002C222A21EB4
:10498500B34006A220921F8002B21F90008BE06008
:1049950012E56C700EA21EB35009A21F302001B3A0
:1049A500B3400280067405900045F0C21EAE55AFB7
:1049B50056AC53AD54EF2DFDEE3CFC74028C068DC8
:1049C500071200398E558F56803AAE55AF56AC5307
:1049D500AD54EF2DFDEE3CFC74018C068D071200E5
:1049E500398E558F56E56CC39402500DAC53AD54BA
:1049F5007410C39D74279C40028009123D8E740675
:104A0500900045F0E55DB41403755D16E55DB423CE
:104A1500127403900045F0D2229000C0E0B4010367
:104A2500123D8EAE57AF58AC53AD54EF2DFDEE3C55
:104A3500FC8C578D58AE53AF54EFD39DEE9C40116F
:104A450090000FE0FAA3E0FBEBC394E8EA9403407F
:104A550002800690000F12623B90000CE0FEA3E07E
:104A6500FFAC53AD54EF2DFDEE3CFC90000CECF08B
:104A7500A3EDF09000C0E0B40118AE53AF54740537
:104A850012622D7401120039900008EEF0A3EFF0C8
:104A95008011AE53AF54740212622D900008EEF0EF
:104AA500A3EFF0C28E758D00758B0075630075548C
:104AB50001755300D28EE55D240875F00984AFF0C9
:104AC5007E00EF4E707590000CE0F8A3E090000AB0
:104AD500C8F0A3C8F090000AE0FEA3E0FFEF4E6027
:104AE5000B7C7B7D8912611B8E518F5290000CE4EB
:104AF500F0A3F0AE51AF527428BE00039F5010E5ED
:104B0500622FFF50010E74011200398E518F5285AC
:104B150052629000C7E0A851B8000DD395524008E5
:104B2500E552900044F080099000C7E014900044DD
:104B3500F0E56C60067552007551009000BEE0B45A
:104B4500030890003DE0655D6002800BA21FB34045
:104B550004D2218002B221E55D640B6005E55DB4F8
:104B65001D099000B0E0600312202B900042E06523
:104B75005D6007900043E0B55D03756E00A213B359
:104B85005006A212B3B34003024C3590007CE0B44A
:104B950001739000FEE0B40214120C5590006FE012
:104BA50075F0BEA4FFAEF08E5B8F5C8056E5667532
:104BB500F00A84FF7E00900576126254E0F55A757E
:104BC5005900AE59AF5A9000A1E012622D74648E5F
:104BD500048F05FF12621D8C5B8D5CE55C90000EF9
:104BE500F0AE59AF5A90007AE012622D74648E04CB
:104BF5008F05FF12621D74BE8C068D0712622D8E05
:104C05005B8F5C801790007AE075F0BEA4FFAEF074
:104C15008E5B8F5C9000A1E090000EF0E560C39480
:104C2500CC500690007AE070028003123E62D213E7
:104C3500E56CB40106E55D640B60028009756F01E2
:104C45009000467401F0E56C70799000C3E0600D4A
:104C550090006EE0A851B800069552400280389049
:104C650000C3E0B4021790003BE0655D600790006B
:104C75003CE0B55D03756F03756B00800CC2007574
:104C85006B00900015E4F0A3F090006EE0600674F0
:104C950009900045F0802C90003BE0655D60079031
:104CA500003CE0B55D03756F0190003BE0B55D0626
:104CB5009000467401F090003CE0B55D06740290EA
:104CC5000046F0A210B3920EA210B330B601B35055
:104CD50003024EA8756D019000A3E0B43D1975E778
:104CE50000A210B34008E5B54404F5B58006E5B566
:104CF50054FBF5B575E710E5B54401F5B5742B9092
:104D05000066F0A210920EE55DD3944A4014D212CB
:104D1500E55DD3946D400B7404900045F0D2227587
:104D25005D469000CBE0B40107E569C394144002E9
:104D35008009123D8E7413900045F0A229300301BD
:104D4500B3501D75E700A229B34008E5B54408F541
:104D5500B58006E5B554F7F5B575E710A2299203B8
:104D6500A22A300401B3501D75E700A22AB34008FA
:104D7500E5B54402F5B58006E5B554FDF5B575E72D
:104D850010A22A9204A22B300501B3500FA22BB317
:104D95004004D2A08002C2A0A22B9205A22C30060C
:104DA50001B3500FA22CB34004D2978002C297A240
:104DB5002C9206A22D300701B3500FA22DB340044B
:104DC500D2A28002C2A2A22D9207A22E300801B360
:104DD500500FA22EB34004D2A18002C2A1A22E92EE
:104DE50008A22F300901B3501D75E700A22FB3406B
:104DF50008E5B54440F5B58006E5B554BFF5B5758C
:104E0500E710A22F9209A230300A01B3501D75E7B1
:104E150000A230B34008E5B54480F5B58006E5B598
:104E2500547FF5B575E710A230920AA231300B0117
:104E3500B3500FA231B34004D2878002C287A2319A
:104E4500920BA232300C01B3500FA232B34004D200
:104E5500908002C290A232920CE569C39441500938
:104E6500740E900045F0123D8E90004DE0FE9000CE
:104E750049E0C39E4009900049E0D3940640097477
:104E8500FB900045F0123D8E900052E060159000B9
:104E950052E0FE90004CE06E600974FE900045F013
:104EA500123D8EA222B34004C296C2959000FBE04B
:104EB500600CAE51AF527414BE00059F400280488D
:104EC500900083E0905BBDF8282873803BA2B4B3C3
:104ED5005005A224B340028005123EBAD224802890
:104EE500A2A3B35005A225B340028005123EBAD253
:104EF500258015A2A4B35005A223B3400280051254
:084F05003EBAD22380028000B5
:105BBD00024ED0024ED2024EE5024EF8024F0B02BB
:025BCD004F0D7A
:104F0D00A215B3B3500890003DE0655D6003024FFC
:104F1D00ECA201B35006A200B3B34003024FE890D8
:104F2D0000BEE0B403028003024FBDA20DB3406783
:104F3D00A221B3402D123615E55CF5FBE55BF5FCC2
:104F4D00D293A202B34002D2879000DCE0B40210EB
:104F5D00123642E55CF5FBE55BF5FC75A700D287E3
:104F6D008033123615E55CF5EBE55BF5ECD291A2DD
:104F7D0002B34006E5B54410F5B59000DCE0B4028F
:104F8D0014123642E55CF5EBE55BF5EC75A700E533
:104F9D00B54410F5B58017123615E55CF5FBE55BEC
:104FAD00F5FCE55CF5EBE55BF5ECD293D291802B4E
:104FBD00123615E55CF5FBE55BF5FCD293A202B369
:104FCD004002D2879000DCE0B40210123642E55C5C
:104FDD00F5FBE55BF5FC75A700D287C215D216A2CD
:104FED0016B3B3500890003EE0655D60030250CBF0
:104FFD00A201B35006A200B3B340030250C7900004
:10500D00BEE0B40302800302509CA20DB34067A220
:10501D0021B3402D123615E55CF5E9E55BF5EAD2D5
:10502D0094A202B34002D2909000DCE0B4021012C0
:10503D003642E55CF5E9E55BF5EA75A700D29080AF
:10504D0033123615E55CF5EDE55BF5EED292A20275
:10505D00B34006E5B54420F5B59000DCE0B402148C
:10506D00123642E55CF5EDE55BF5EE75A700E5B5AD
:10507D004420F5B58017123615E55CF5E9E55BF5CD
:10508D00EAE55CF5EDE55BF5EED294D292802B125C
:10509D003615E55CF5E9E55BF5EAD294A202B3407D
:1050AD0002D2909000DCE0B40210123642E55CF5BD
:1050BD00E9E55BF5EA75A700D290D215C216E56F4A
:0E50CD00905BCFF828287302551C9000E3E09A
:065BCF000250D40250D781
:1050DB00905C02F8282873121B078012121B0780A2
:0E50EB000D121B918008121C3D8003121C3D0B
:0F5C02000250E20250E70250EC0250F10250F65D
:1050F900756F0202551C121D69121E80A237B3403A
:10510900229000A5E0F56B900076E0256BFE9000FB
:1051190044E075F01E84FC7F00EE2CF53474109089
:105129000045F09007AEE0FEA3E0FF740A12622D7D
:1051390090000AE0FCA3E0FD74098F02FF12621DD2
:105149008D078C038E048A058B0612611B9007B2AA
:10515900EEF0A3EFF074F0BE00039F500B74F090D3
:1051690007B2F8E4F0E8A3F0E53470037534019070
:1051790007B2E0FEA3E0FFE5342FFF50010E9007D0
:0D518900B2EEF0A3EFF0756F03900046E06A
:035BD5000250FF7C
:10519600905C11F82828738010A2384003756F0AB6
:0951A6008007A2384003756F0B6D
:095C110002519D02519F0251A8AD
:1051AF0002551C9006BDE060031221149000FCE034
:1051BF00B401149000FDE0A851B8000495525007B7
:1051CF00E55EC3955F4002800302525C9000B1E040
:1051DF00D39402403F900085E02403A851B8000407
:1051EF0095525009900087E0D3956050028008D205
:1051FF00017408900045F0900085E0A851B80005B3
:10520F00D39552500B900087E02403C39560500252
:10521F00C2018039900085E02403A851B80004959D
:10522F00525007E55EC3955F40028008D2017408B3
:10523F00900045F0900085E0A851B80005D3955235
:10524F005009E55F240FC3955E5002C2019000CB59
:10525F00E07007E569C3941440028002D201A201F5
:10526F004005756F04800A756F10900015E4F0A368
:10527F00F0A20DB34029E56675F00A84FF7E009019
:10528F000576126254E0C394695005122060800FB6
:10529F009007B0E0F8A3E09007AEC8F0A3C8F00203
:0652AF00551C9000B1E067
:065BD8000251B20252B1BD
:1052B500905C1AF8282873120D3F8012120D3F805A
:0E52C5000D120EED8008120F9F8003120F9F36
:0F5C1A000252BC0252C10252C60252CB0252D0F9
:1052D3009006C1E060031221F0756F0502551C12A0
:1052E30010AB756F069006C5E060031222E09006CE
:1052F300C9E060031223BC02551C90000EE0600657
:10530300A20DB3B34002801D90000EE02529FFAE2D
:105313002850010E8E288F29E55DD39412500690F4
:10532300000EE014F01212F1756F079006CDE060E5
:10533300031224989006D1E0600312257402551CD1
:105343009000FEE0B40203120CCD12154E756F08E7
:105353009006D5E060031226509006D9E060031250
:10536300272C02551C12190AA215B35005A216B315
:1053730040028004D215D216756F109006DDE060EE
:10538300031228089006E1E060031228E402551C8A
:1053930002551C900035E0C394465008C2967446EB
:1053A300900035F090003FE0B4011DE534240AF588
:1053B300349007B2E0FEA3E0FF740A2FFF50010E02
:1053C3009007B2EEF0A3EFF090003FE0B4021DE5CA
:1053D300342414F5349007B2E0FEA3E0FF74142FD5
:1053E300FF50010E9007B2EEF0A3EFF085345A752B
:1053F300590090003BE0F57212368DE55C90003564
:10540300F0900004E559F0A3E55AF0E572900036F8
:10541300F0C2189007B2E0F559A3E0F55A90003BAB
:10542300E0F57212368DE55C900033F0900000E5F4
:1054330059F0A3E55AF0E572900034F0C217E56C19
:10544300B40105756F0B8003756F0302551C900043
:1054530039E0C3944650139000CCE0B40104C296E3
:105463008002C2957446900039F0900040E0B40188
:105473001DE534240AF5349007B2E0FEA3E0FF747F
:105483000A2FFF50010E9007B2EEF0A3EFF0900049
:1054930040E0B4021DE5342414F5349007B2E0FE75
:1054A300A3E0FF74142FFF50010E9007B2EEF0A398
:1054B300EFF085345A75590090003CE0F5721236CE
:1054C3008DE55C900039F0900006E559F0A3E55AAC
:1054D300F0E57290003AF0C21A9007B2E0F559A3D2
:1054E300E0F55A90003CE0F57212368DE55C9000D1
:1054F30037F0900002E559F0A3E55AF0E572900009
:1055030038F0C219E56CB40103756C00756F038044
:095513000880068004800280007B
:105BDE000252E20252FD02534302536802539302F1
:105BEE005396025451025514025516025518025579
:045BFE001A02551C16
:10551C00900033E0B55D0280030255BEA2174072C5
:10552C00900000E0FEA3E0FFEF4E6021AE55AF56B9
:10553C00900000E0FCA3E0FD120003740A8E048FBF
:10554C0005FF12621D900000ECF0A3EDF09000340A
:10555C00E0601A900000E0FEA3E0FFAC55AD56EF02
:10556C002DFDEE3CFC900000ECF0A3EDF09000342F
:10557C00E0D39401401A900000E0FEA3E0FFAC558C
:10558C00AD56EF2DFDEE3CFC900000ECF0A3EDF0E1
:10559C00D217AE53AF54900000E0FCA3E0FDEFC374
:1055AC009DEE9C400D123F07D296C21774C8900016
:1055BC0033F0A217B3B35007900033E0B55D02800F
:1055CC000D123F07D29674C8900033F0C2179000AA
:1055DC0035E0B55D028003025679A2184072900046
:1055EC0004E0FEA3E0FFEF4E6021AE55AF569000F5
:1055FC0004E0FCA3E0FD120003740A8E048F05FF87
:10560C0012621D900004ECF0A3EDF0900036E06007
:10561C001A900004E0FEA3E0FFAC55AD56EF2DFD53
:10562C00EE3CFC900004ECF0A3EDF0900036E0D3DF
:10563C009401401A900004E0FEA3E0FFAC55AD5677
:10564C00EF2DFDEE3CFC900004ECF0A3EDF0D21835
:10565C00AE53AF54900004E0FCA3E0FDEFC39DEE0D
:10566C009C400AC2967446900035F0C218A218B33A
:10567C00B35007900035E0B55D02800AC2967446BF
:10568C00900035F0C218900037E0B55D028003023F
:10569C005734A2194072900002E0FEA3E0FFEF4ED7
:1056AC006021AE55AF56900002E0FCA3E0FD120065
:1056BC0003740A8E048F05FF12621D900002ECF039
:1056CC00A3EDF0900038E0601A900002E0FEA3E039
:1056DC00FFAC55AD56EF2DFDEE3CFC900002ECF00E
:1056EC00A3EDF0900038E0D39401401A900002E052
:1056FC00FEA3E0FFAC55AD56EF2DFDEE3CFC90004B
:10570C0002ECF0A3EDF0D219AE53AF54900002E0CE
:10571C00FCA3E0FDEFC39DEE9C400D123F07D2951C
:10572C00C21974C8900037F0A219B3B35007900097
:10573C0037E0B55D02800D123F07D29574C890001A
:10574C0037F0C219900039E0B55D0280030257EFC3
:10575C00A21A4072900006E0FEA3E0FFEF4E60211B
:10576C00AE55AF56900006E0FCA3E0FD12000374AA
:10577C000A8E048F05FF12621D900006ECF0A3ED5B
:10578C00F090003AE0601A900006E0FEA3E0FFAC57
:10579C0055AD56EF2DFDEE3CFC900006ECF0A3ED64
:1057AC00F090003AE0D39401401A900006E0FEA37A
:1057BC00E0FFAC55AD56EF2DFDEE3CFC900006EC39
:1057CC00F0A3EDF0D21AAE53AF54900006E0FCA358
:1057DC00E0FDEFC39DEE9C400AC2957446900039E3
:1057EC00F0C21AA21AB3B35007900039E0B55D02AB
:1057FC00800AC2957446900039F0C21A9000CEE02F
:10580C00B402028003025924900068E0D3956550DD
:10581C0064900068E0F4042565FE9000D1E08E00F1
:10582C00F5F0E884FF7E008F72EFC39410500CEFFC
:10583C008572F0A4FDACF08D7280037572FF900040
:10584C0068E0D39572400B900068E0C39572F570D8
:10585C0080037570009000ECE0D3957040069000CA
:10586C00ECE0F5709000EDE0C3957050069000ED03
:10587C00E0F5708071900068E0C39565FE9000D1F2
:10588C00E08E00F5F0E884FF7E008F72EFC3941079
:10589C00500CEF8572F0A4FDACF08D728003757224
:1058AC00FF85725A755900900068E0255AFFAE5971
:1058BC0050010E8E598F5A74FFBE0009D39F4005BC
:1058CC00855A7080037570FF9000ECE0D3957040A2
:1058DC00069000ECE0F5709000EDE0C3957050067A
:1058EC009000EDE0F570A20DB3B3500D900069E09F
:1058FC00FE9000D9E0D39E5002800A7407900045B8
:10590C00F0C2A2801375A710E5CDC395704004C2F8
:10591C00A28002D2A275A700E56EC39409500AA218
:10592C00EDB34005C2ED122C7AAE53AF547410C3D4
:10593C009F74279E400C900067E0C3945A4003026A
:10594C005B96A212B34009123D8E7406900045F08E
:10595C00A21DB34008E5B54404F5B58006E5B55481
:10596C00FBF5B5A214B3500EE560D394334007E5B4
:10597C0060C394CC4002802FE5B54401F5B5742B7F
:10598C00900066F090007AE075F0BEA4FFAEF08E49
:10599C005B8F5C7402BE000AD39F4006755C027577
:1059AC005B00123E62D214900067E0D39401400772
:1059BC00E560C3941A40028002C2149006BDE060F8
:1059CC0003122114A229300301B35017A229B340AA
:1059DC0008E5B54408F5B58006E5B554F7F5B5A26C
:1059EC002992039006C1E060031221F0A22A300430
:1059FC0001B35017A22AB34008E5B54402F5B580AF
:105A0C0006E5B554FDF5B5A22A92049006C5E060F2
:105A1C00031222E0A22B300501B3500FA22BB3408E
:105A2C0004D2A08002C2A0A22B92059006C9E0600D
:105A3C00031223BCA22C300601B3500FA22CB3408E
:105A4C0004D2978002C297A22C92069006CDE060F9
:105A5C0003122498A22D300701B3500FA22DB3408E
:105A6C0004D2A28002C2A2A22D92079006D1E060BD
:105A7C0003122574A22E300801B3500FA22EB3408E
:105A8C0004D2A18002C2A1A22E92089006D5E06099
:105A9C0003122650A22F300901B35017A22FB34086
:105AAC0008E5B54440F5B58006E5B554BFF5B5A29B
:105ABC002F92099006D9E0600312272CA230300AED
:105ACC0001B35017A230B34008E5B54480F5B5805A
:105ADC0006E5B5547FF5B5A230920A9006DDE0607C
:105AEC0003122808A231300B01B3500FA231B3407E
:105AFC0004D2878002C287A231920B9006E1E0604B
:105B0C00031228E4A232300C01B3500FA232B3407E
:105B1C0004D2908002C290A232920C900067E0C333
:105B2C00945A5010E56EB40909900067E004F075C2
:105B3C006E00803BE56EB40903756E0075540075FC
:105B4C005300758D00758B00756300900066E0C383
:105B5C0094415008900066E004F080067441900077
:105B6C0066F0900066E0B44106E5B554FEF5B590DC
:105B7C000067E0D394014007E569C394414002807B
:0D5B8C0009740E900045F0123D8E02466532
:105C29000000010001400160018001A001C001E004
:105C390002000300039603B603D603F4040005002B
:105C49000512052405360548055A056C057E05909B
:105C590005A805C005DE0600061406280646066ED8
:105C690006AE00FF013F015F017F019F01BF01DF18
:105C790001FF02FF039503B503D503F303FF04FFF7
:105C890005110523053505470559056B057D058F63
:105C990005A705BF05DD05F1061306270645066DAF
:105CA90006AD06ED0FAA0FA50F9F0F9A0F940F8D42
:105CB9000F870F800F780F710F680F600F570F4E06
:105CC9000F450F3B0F300F250F1A0F0E0F020EF560
:105CD9000EE80EDB0ECC0EBE0EAE0E9F0E8E0E7DA6
:105CE9000E6C0E5A0E470E340E200E0C0DF70DE2F7
:105CF9000DCB0DB50D9D0D850D6D0D540D3A0D2076
:105D09000D050CE90CCE0CB10C940C760C580C3A20
:105D19000C1B0BFB0BDB0BBB0B9A0B790B570B35D6
:105D29000B130AF10ACE0AAB0A870A640A400A1C55
:105D390009F809D409B0098C09670943091F08FB47
:105D490008D608B2088E086A0846082307FF07DC48
:105D590007B9079607730751072F070D06EC06CAFF
:105D690006AA068906690649062A060A05EC05CD2A
:105D790005B0059205750558053C0520050504EA99
:105D890004CF04B5049C0482046904510439042233
:105D9900040B03F403DE03C803B2039D03890375EF
:105DA9000361034D033B03280316030402F202E1D6
:105DB90002D102C002B002A00291028202730265FE
:105DC90002570249023C022F02220216020901FD72
:105DD90001F201E601DB01D001C601BB01B101A756
:105DE900019D0194018B01820179017001680160B3
:105DF900015801500148014101390132012B0125A6
:105E0900011E01180111010B010500FF00FA0FA67F
:105E19000FA00F990F920F8B0F840F7C0F740F6BCC
:105E29000F620F580F4E0F430F380F2C0F1F0F1211
:105E39000F050EF70EE80ED80EC80EB70EA50E9375
:105E49000E800E6C0E580E420E2C0E150DFD0DE433
:105E59000DCB0DB10D950D790D5D0D3F0D200D018A
:105E69000CE10CC00C9E0C7C0C590C350C100BEA87
:105E79000BC40B9E0B760B4F0B260AFD0AD40AAAFC
:105E89000A800A550A2A09FF09D409A8097C095078
:105E9900092508F908CD08A10875084A081E07F35D
:105EA90007C8079D07730749072006F706CE06A608
:105EB900067E06570630060A05E405BF059B0577E9
:105EC90005540532051004EF04CE04AE048F0471A5
:105ED90004530435041903FD03E203C703AD039416
:105EE900037B0363034B0334031E030802F302DE3F
:105EF90002CA02B602A30291027F026D025C024C41
:105F0900023C022C021D020E020001F201E401D73B
:105F190001CA01BE01B101A6019A018F0185017A69
:105F290001700166015D0153014A014101390131E5
:105F39000129012101190112010B010400FD00F7DA
:105F490000F000EA00E400DE00D900D300CE00C969
:105F590000C400BF00BA00B500B100AD00A800A49C
:105F690000A0009C009900950091008E008A00878E
:085F790000840081007E007B22
:10009E007547009007BAE4F0A3F075310075300093
:1000AE00754D00754E00C234D23574FE9007C4F8FB
:1000BE00E4F0E8A3F074FE9007C6F8E4F0E8A3F0CD
:1000CE00745A9007C8F0745A9007C9F0D236C228F5
:1000DE00C238C23322750B00750A00AE0AAF0BACE4
:1000EE0008AD09EDC39FEC9E401674FF12620D75AC
:1000FE00CF01780B740126F6500418E436F650DB67
:10010E0022900041E0B4AA1C900776E0B43C159012
:10011E0007B6E0FEA3E0FFEF4E6009741EBE0004BA
:10012E00D39F500302023D755C00755B0075F809A4
:10013E009007B6E0FEA3E0FF74076F4E6006740EE4
:10014E006F4E7006743A900776F09007B6E0FEA3F5
:10015E00E0FF7408BE001ED39F401A7E017F0890F8
:10016E0007B6E0FCA3E0FD1DBDFF011C1200038ECF
:10017E00598F5A801F9007B6E0FEA3E0FF74081255
:10018E0062718F048E057E017F08CDCCCD120003E7
:10019E008E598F5AAE5BAF5C740CD39F74019E5018
:1001AE0003020238A2F9B3407EE55C455B7003752D
:1001BE00A382AE5BAF5C74016F4E700375A300AE8D
:1001CE005BAF5C74026F4E700D9007B7E075F00276
:1001DE00A4FDACF08DA3AE5BAF5C74036F4E7003E9
:1001EE0075A300AE5BAF5C7403BE00039F5013ACEF
:1001FE0059AD5AED2FFFEC3EFE900072126254E0A4
:10020E00F5A3AE5BAF5CEFB40B09EEB4010574144D
:10021E0012620DAE5BAF5CEFB40B07EEB40103756B
:10022E00F80D785B1262810201A2900041E4F02287
:10023E00755C00755B0075F8099007B6E0FEA3E0EB
:10024E00FF7408BE001ED39F401A7E017F089007E0
:10025E00B6E0FCA3E0FD1DBDFF011C1200038E598C
:10026E008F5A801F9007B6E0FEA3E0FF740812625B
:10027E00718F048E057E017F08CDCCCD1200038ECA
:10028E00598F5AAE5BAF5C7411D39F74019E5003AD
:10029E0002036EA2F9B3500302036BE55C455B707B
:1002AE000375A3D2AE5BAF5C74016F4E700375A382
:1002BE0000AE5BAF5C74026F4E700D9007B7E075C9
:1002CE00F002A4FDACF08DA3AE5BAF5C74036F4E79
:1002DE00700375A300AE5BAF5C74046F4E70037554
:1002EE00A300AE5BAF5C74056F4E700375A300AEDA
:1002FE005BAF5C74066F4E700375A300AE5BAF5CB4
:10030E0074076F4E700375A300AE5BAF5C74086F1D
:10031E004E700375A300AE5BAF5C7408BE00039F06
:10032E005016AC59AD5AED2FFFEC3EFE90006D12FB
:10033E006254E5A3F075A300AE5BAF5CEFB4100999
:10034E00EEB40105741412620DAE5BAF5CEFB41027
:10035E0007EEB4010375F80D785B1262810202910B
:10036E0022755C00755B0075F809AE5BAF5C7417A7
:10037E00BE0004D39F5003020447A2F9B3500302F8
:10038E000444E55C455B700375A3D2AE5BAF5C7451
:10039E00016F4E700375A300AE5BAF5C74026F4EBF
:1003AE00700D9007B7E075F002A4FDACF08DA3AE12
:1003BE005BAF5C74036F4E700375A300AE5BAF5CF6
:1003CE0074046F4E700375A300AE5BAF5C74056F63
:1003DE004E700375A300AE5BAF5C74066F4E700378
:1003EE0075A300AE5BAF5C74076F4E700375A30010
:1003FE00AE5BAF5C74086F4E700375A300AE5BAF5F
:10040E005C7408BE00039F500C90004F126254E5BE
:10041E00A3F075A300AE5BAF5C74166F4E700574DF
:10042E001412620DAE5BAF5C74166F4E700375F8EE
:10043E000D785B12628102037822900041E0B4AB2A
:10044E000280030204E2755C00755B0075F809AE6C
:10045E005BAF5C7412BE007CD39F4078A2F9B340B0
:10046E0070E55C455B700375A382AE5BAF5C740197
:10047E006F4E700375A300AE5BAF5C74026F4E706F
:10048E000D9007B7E075F002A4FDACF08DA3AE5B46
:10049E00AF5C74036F4E700375A300AE5BAF5C74FC
:1004AE0003BE00039F5009900054126254E0F5A35E
:1004BE00AE5BAF5C74116F4E7005741412620DAEAC
:1004CE005BAF5C74116F4E700375F80D785B126242
:1004DE008102045D229007C1E4F074649007B6F8BF
:1004EE00E4F0E8A3F012036F74C89007B6F8E4F0D6
:1004FE00E8A3F090005BE0B4371A900058E090004B
:10050E004FF0900059E0900050F090005AE09000AB
:10051E0051F080469007C17401F074659007B6F8EB
:10052E00E4F0E8A3F012036F74C89007B6F8E4F095
:10053E00E8A3F090005BE0B4371A900058E090000A
:10054E004FF0900059E0900050F090005AE090006B
:10055E0051F0800674029007C1F09007C2E4F07467
:10056E00669007B6F8E4F0E8A3F012036F74C89033
:10057E0007B6F8E4F0E8A3F090005AE0B437129012
:10058E000058E0900049F0900059E0900052F08041
:10059E00769007C27401F074679007B6F8E4F0E83D
:1005AE00A3F012036F74C89007B6F8E4F0E8A3F056
:1005BE0090005AE0B43712900058E0900049F09045
:1005CE000059E0900052F0803E74029007C2F07421
:1005DE00689007B6F8E4F0E8A3F012036F74C890C1
:1005EE0007B6F8E4F0E8A3F090005AE0B4371290A2
:1005FE000058E0900049F0900059E0900052F080D1
:10060E000674039007C2F022E54E64046006E59975
:10061E0064FF6002802AA2344004D2348020E54E6A
:10062E00600874E6254E900045F0754E00E54D606D
:10063E000874F0254D900045F0754D00C2348002CF
:10064E00C234E54E9033F8F8282873754E00E599BC
:10065E00B4FF03754D01E599B4FE03754D02E5999E
:10066E00B4FD03754D03E599B4FC03754D04E5998E
:10067E00B4FA03754D05E599B4FB06754E01123DAE
:10068E008EE599B4F906754E04123D8EE599D39414
:10069E00E54007E599C394F04002801685994F75A1
:1006AE004E027E017F00E54FC394E612622D8E321C
:1006BE008F339007BAE4F0A3F0E599D394C44007C2
:1006CE00E599C394E64002802885994F754E0374D0
:1006DE00E5C3954FF533753200AE32AF33905C29DA
:1006EE001261FCE493F87401939007BAC8F0A3C8A2
:1006FE00F0D299020AB3900058E070429007BAE027
:10070E00FEA3E0FF74FFBE00039F5009EFC39446A3
:10071E00EE940640119007BAE0FEA3E0FFEFD394EB
:10072E006DEE940640139007BAE0FEA3E0FF900032
:10073E0076126254E599F0800385997380119007C3
:10074E00BAE0FEA3E0FF900076126254E599F090B5
:10075E0007BA12623B9007BAE0FEA3E0FFEFB401C6
:10076E0006EEB40702800302089B900776E0B43CC5
:10077E00028003020885C29C900058E0900114F09C
:10078E00900059E0900083F090005AE09000A3F0A2
:10079E0090005BE09000CCF090005CE0900078F070
:1007AE0090005DE09000BEF090005EE09000DCF006
:1007BE0090005FE09000B0F0900060E09000CEF00E
:1007CE00900061E09000FEF012377290006AE090A7
:1007DE0000E5F090006BE090009CF090006CE090D3
:1007EE00009DF074639007B6F8E4F0E8A3F074ABE4
:1007FE00900041F0120448900041E4F075096475D0
:10080E0008001200E3A21C4038757201E572D39401
:10081E0007502CE5729007B6F8E4F0E8A3F074AA3E
:10082E00900041F012010FE572C39407500975094B
:10083E00647508001200E37872740126F650CD80BC
:10084E0036757208E572D3940E502CE5729007B689
:10085E00F8E4F0E8A3F074AA900041F012010FE55D
:10086E0072C3940E50097509647508001200E3787E
:10087E0072740126F650CD74C89007B6F8E4F0E80D
:10088E00A3F0D29C754E00754D007599FB020AB30C
:10089E009007BAE0FEA3E0FFEF4E70068599317522
:1008AE0030009007BAE0FEA3E0FF74016F4E701B9C
:1008BE00AC30AD31AA32AB33ED2BFBEC3AFA8A06F3
:1008CE008B07900076126254E599F09007BA126287
:1008DE003B9007BAE0FEA3E0FF74026F4E7021ACAE
:1008EE0030AD3174566D4C7006E54F64E660028093
:1008FE0003123D8E123772854F99754E00754D005D
:10090E00020AB39007BAE0FEA3E0FF9000761262EF
:10091E0054E599F09007BA12623B9007BAE0FEA335
:10092E00E0FFAC32AD338F028E038C068D07905CE8
:10093E006B1261FCE493F9740193FEEAD39EEB997A
:10094E004009854F99754E00754D00020AB3900708
:10095E00BAE0FEA3E0FF900076126254E599F090A3
:10096E0007BA12623B9007BAE0FEA3E0FFEFB400B5
:10097E0006EEB401028003020AB3900051E075F056
:10098E0002A4FDACF08D72ED90007612625FEDFA6E
:10099E00E0FBEA90007912625FEBFAE0FBEA2BFAD9
:1009AE00900051E0B502028003020AA50DED900001
:1009BE007612625FE572FDE0FAED90007A12625FE8
:1009CE00EAFDE0FAEDC39AFD900051E0B505028014
:1009DE0003020AA5E57290007812625FE572FDE0EF
:1009EE00FAED90007B12625FEAFDE0FAED2AFD90CF
:1009FE000051E0B505028003020AA5E57290007C65
:100A0E0012625FFDE0FAED900051E0F4042A9000CE
:100A1E0058F0E57290007D12625FFDE0FAED9000F5
:100A2E0051E0F4042A900059F0E57290007E1262B3
:100A3E005FFDE0FAED900051E0F4042A90005AF0C8
:100A4E00E57290007F12625FFDE0FAED900051E0DA
:100A5E00F4042A9007B6F8E4F0E8A3F074AB900023
:100A6E0041F01204487509647508001200E39007FE
:100A7E00B612623B1204487509647508001200E351
:100A8E009007B612623B1204487599F975096475A0
:100A9E0008001200E380FE7599FF75096475080061
:050AAE001200E380FED0
:0F33F80002065902070402089E02091102095C2D
:100AB30022E54D903407F8282873020B989007BA63
:100AC300E0FEA3E0FF900047126254E0F59990071F
:100AD300BA12623B9007BAE0FEA3E0FF74116F4EB7
:100AE3007003754D00020B98856D99020B98900762
:100AF300BAE0FEA3E0FF900076126254E0F599EFAE
:100B0300B40107EEB40703754D009007BA12623BB8
:070B1300020B989007BBE004
:0F340700020ABD020AC0020AEB020AF1020B160A
:100B1A009035BAF82828738552998067855E99803E
:100B2A0062856099805D856499805885669980534D
:100B3A00856799804E85689980498569998044902E
:100B4A000016E0F599803CA235B340077599FAC2C0
:100B5A00358017A226B3400575990F800B90004582
:100B6A00E0F599900045E4F0C2268017856A9980DD
:100B7A0012856599800D856B9980087599FC8003AB
:030B8A00754D00A6
:1035BA00020B21020B26020B2B020B30020B3502E7
:1035CA000B3A020B3F020B44020B49020B51020B4E
:0D35DA0076020B7B020B80020B85020B8A30
:0B0B8D009007BA12623B80031235E7AC
:03341600020B9511
:100B980022E537255AFFAE5950010E9000761262B1
:100BA80054E0F538E537255AFFAE5950010E0FBF0E
:100BB80000010E900076126254E0F539853F3BE55E
:100BC80038B539058538378041E539D39538401D22
:100BD800E539C39538853AF0A4FFAEF0E53B8E04BD
:100BE8008F05FF12621DED2538F537801DE538C3E6
:100BF8009539853AF0A4FFAEF0E53B8E048F05FFEA
:100C080012621DEDF4042538F53722E539D39538FD
:100C1800401DE539C39538853AF0A4FFAEF0E53BB1
:100C28008E048F05FF12621DED2538F537801DE50E
:100C380038C39539853AF0A4FFAEF0E53B8E048FB2
:100C480005FF12621DEDF4042538F5372290007C6B
:100C5800E0B40170E56675F00A84FF7E008F37E521
:100C68006675F00A84ADF07C008D3A753F0A7559B7
:100C780005755A24E537C394115005120B9980065F
:100C88009005ABE0F537E53790006FF0E56675F055
:100C98000A84FF7E008F37E56675F00A84ADF07C24
:100CA800008D3A753F0A755905755A5AE537C39448
:100CB800115005120B9980069005E1E0F537E537EC
:100CC80090000EF02290007CE0B4016AE56675F0B1
:100CD8000A84FF7E008F37E56675F00A84ADF07CE4
:100CE800008D3A753F0A755905755A36E537C3942C
:100CF800115005120B9980069005BDE0F537853730
:100D08004BE56675F00A84FF7E008F37E56675F05F
:100D18000A84ADF07C008D3A753F0A755905755AFD
:100D280048E537C394115005120B9980069005CFFA
:100D3800E0F53785374C22E55E75F00484FF7E00C8
:100D48008F37E55E75F00484ADF07C008D3A753F11
:100D580004755901755A00E537C3943F5005120BC5
:100D68009980069001B5E0F53785372975280090F8
:100D78000044E075F020A4FFAEF09000C7E08E04B8
:100D88008F05FF12621D8D379000AFE0D3955E503E
:100D980003020E459000D3E0D3955E4010ED90011C
:100DA800B612625FE0F52B752A00020E4290009E93
:100DB800E0D3955E4043E5379001B612625FE0F5F7
:100DC80038E5379001D612625FE0F5399000D3E03C
:100DD800F404255EF53A90009EE0FE9000D3E0F41E
:100DE800042EF53BE538B539058538378003120CF4
:100DF8001385372B752A008041E5379001D612629A
:100E08005FE0F538E5379001F612625FE0F539905A
:100E1800009EE0F404255EF53A9000AFE0FE9000F5
:100E28009EE0F4042EF53BE538B539058538378062
:100E380003120C1385372B752A00020EEC9000D68E
:100E4800E0D3955E5011E53790023612625FE0F507
:100E58002B752A00020EEC90009FE0D3955E50435C
:100E6800E53790021612625FE0F538E537900236F2
:100E780012625FE0F53990009FE0F404255EF53AD0
:100E88009000D6E0FE90009FE0F4042EF53BE53894
:100E9800B539058538378003120C1385372B752A29
:100EA800008041E5379001F612625FE0F538E537DA
:100EB80090021612625FE0F5399000AFE0F4042565
:100EC8005EF53A90009FE0FE9000AFE0F4042EF546
:100ED8003BE538B539058538378003120C1385375B
:100EE8002B752A00229000E7E0F53C753F117559F3
:100EF80002755A00AE51AF52E53C75F00FA4FDAC37
:100F0800F0EDD39FEC9E4021E53C8E048F05FF1247
:100F1800621DED75F010A4FFAEF0E55E75F011846A
:100F2800FD7C00ED2FF53D800EE55E75F01184FF28
:100F38007E00EF24F0F53D853D37E55E75F01184C0
:100F4800AFF07E008F3A120B9985373EAE51AF5203
:100F58009000E7E075F00FA4FDACF0EDD39FEC9E98
:100F68004028755902755A10853D37120B99853EF0
:100F780038853739AE51AF52E53C8E048F05FF12E4
:100F880062488D3A853C3B120C1385372975280039
:100F9800752B64752A00229000E7E0F53C753F1137
:100FA800755902755A00AE51AF52E53C75F00FA461
:100FB800FDACF0EDD39FEC9E4021E53C8E048F05FF
:100FC800FF12621DED75F010A4FFAEF0E56075F03C
:100FD8001184FD7C00ED2FF53D800EE56075F01164
:100FE80084FF7E00EF24F0F53D853D37E56075F020
:100FF8001184AFF07E008F3A120B9985373EAE51BF
:10100800AF529000E7E075F00FA4FDACF0EDD39F70
:10101800EC9E4028755902755A10853D37120B9978
:10102800853E38853739AE51AF52E53C8E048F0581
:10103800FF1262488D3A853C3B120C13853729759F
:1010480028009000B1E0B40453E55E75F00484FF15
:101058007E008F37E55E75F00484ADF07C008D3A34
:10106800753F04755901755A00E537C3943F50051B
:10107800120B9980069001B5E0F537AE28AF29E547
:101088003712622D74648E048F05FF12621DAE281C
:10109800AF29EF2DFDEE3CFC8C288D29752B64754E
:1010A8002A002290007CE0B40146E56675F00A84C7
:1010B800FF7E008F37E56675F00A84ADF07C008D01
:1010C8003A753F0A755905755A00E537C3941150AA
:1010D80005120B998006900587E0F537AE2AAF2BED
:1010E800E5372FFF50010E74641262718E2A8F2B20
:1010F80090007DE0B40146E56775F00A84FF7E0044
:101108008F37E56775F00A84ADF07C008D3A753F3E
:101118000A755905755A6CE537C394115005120BB9
:101128009980069005F3E0F537AE2AAF2BE5372F07
:10113800FF50010E74641262718E2A8F2B90008CFE
:10114800E0B40249E569C3944175F00584FF7E0067
:101158008F37E56975F00584ADF07C008D3A753FF1
:1011680005755906755A00E537C394135005120BD7
:10117800998006900689E0F537AE2AAF2BE5372F20
:10118800FF50010E74641262718E2A8F2B9000CE6C
:10119800E0B40202800302124AE55E75F01584FF8E
:1011A8007E008F37E55E75F01584ADF07C008D3AD2
:1011B800753F15755903755AF4E537C3940B5005F7
:1011C800120B998006900475E0F537E53775F0FF46
:1011D800A4FFAEF09000CFE08E048F05FF12621DD1
:1011E800ED900068F0E56575F078A4FFAEF074FF47
:1011F8008E048F05FF12621D8C598D5A74028C065D
:101208008D071200398F37AC59AD5A7404FF12623A
:10121800488D3A753F04755906755A28E537C394C1
:101228001D5005120B9980069006BBE0F537AE2AD3
:10123800AF2BE5372FFF50010E74641262718E2AAE
:101248008F2B90007BE0B4025DE56075F064A4FF2D
:10125800AEF074081200398E5B8F5C74058E048FB3
:1012680005FF12621D8D37AE5BAF5C74058E048F6F
:1012780005FF1262488D3A753F05755905755ADEA6
:10128800E537C394135005120B998006900667E062
:10129800F537AE2AAF2BE5372FFF50010E746412D5
:1012A80062718E2A8F2B9000BDE0703C900044E064
:1012B80075F00584FF7E008F37900044E075F005D7
:1012C80084ADF07C008D3A753F05755905755AC097
:1012D800E537C3941D5005120B998006900653E01C
:1012E800F537E537900070F022900084E0B40117DC
:1012F8009007BDE0252BFFAE2A50010E9000D8E0E4
:101308001262718E2A8F2B9000FCE0B401149000B9
:10131800FDE0A851B8000495525007E55EC3955FFB
:10132800400280129000A6E0252BFFAE2A50010E45
:101338008E2A8F2B802F900084E0B40316A228B346
:10134800B350109007C0E0C39405A851B8000695A3
:1013580052400280109000A6E0252BFFAE2A5001D3
:101368000E8E2A8F2B90007EE0B4020280030215B5
:101378004D900081E0602FE566D3944640289000A8
:101388000FE0FEA3E0FF9000BCE075F003A4FDAC05
:10139800F0EFD39DEE9C400E9000E0E0A851B8001D
:1013A80005D39552500302154D9000C9E0855EF0B3
:1013B800A4FFAEF0740512622D74071200398E591D
:1013C8008F5A900088E0A851B800049552501290A6
:1013D8000089E075F002A4FDACF0EFC39DEE9C40DF
:1013E8000302154DE55E75F00B84FF7E009006063E
:1013F800126254FEE0FFEE900080E0FEEF8E00885F
:10140800F0A4FFAEF074648E048F05FF12621D8C89
:10141800598D5A900044E075F018A4FFAEF0900082
:10142800C7E08E048F05FF12621D8C068D0790069B
:101438001E126254AE59AF5AE012622D74648E04C3
:101448008F05FF12621D8C598D5AE564A859B800A2
:1014580077D3955A4072E564C3955AFFE49559FECF
:101468008E598F5A7428BE00039F500C755A2875E0
:101478005900740D900045F0AE59AF5A900081E0C4
:1014880012622D74288E048F05FF12621D8C598DEF
:101498005AAE28AF29740A8E048F05FF12621D8D7B
:1014A800068C07AC59AD5ACFCECF120003740A8E02
:1014B800048F05FF12621D8C598D5AAE28AF291270
:1014C80062798E288F29807DE564A859B800049533
:1014D8005A5072AE59AF5AE5641262718E598F5ADA
:1014E8007428BE00039F500C755A28755900740D56
:1014F800900045F0AE59AF5A900081E012622D7409
:10150800288E048F05FF12621D8C598D5AAE28AFA4
:1015180029740A8E048F05FF12621D8D068C07AC94
:1015280059AD5ACFCECF120003740A8E048F05FF2F
:1015380012621D8C598D5AAE28AF29EF2DFDEE3C55
:10154800FC8C288D29229000DCE0B4026AE55E75E7
:10155800F00884FF7E008F37E55E75F00884ADF0F3
:101568007C008D3A753F08755901755AE0E537C317
:10157800943F5005120B998006900275E0F5378567
:10158800372D752C00AE2CAF2DAC2AAD2B120003D5
:1015980074648E048F05FF12621D8C2C8D2D9000B3
:1015A80079E08C068D0712622D74648E048F05FF16
:1015B80012621D8C2C8D2DAE28AF29AC2AAD2B12B2
:1015C800000374648E048F05FF12621D8C288D2918
:1015D800900079E08C068D0712622D74648E048F5A
:1015E80005FF12621D8C288D29A20D401DAE51AF3A
:1015F800527405BE00039F5002D20DE560D394CC0F
:101608004008D2017411900045F09000DBE0B4026C
:10161800089000DDE0640160028035AE28AF29E55E
:101628006A12622D74E78E048F05FF12621D8C28E2
:101638008D299000DCE0B40217AE2CAF2DE56A12BC
:10164800622D74E78E048F05FF12621D8C2C8D2D80
:1016580090009BE05402601B900092E0A851B800F3
:1016680012D39552400DA20DB3B35007E560C39451
:101678009A40028028AE35AF36900090E075F002AF
:10168800A4FDACF0EF2DFDEE3CFC74022DFD5001E5
:101698000CE560BC0007D39D4003754301856036A7
:1016A800753500E54370030217919000EEE0C3958D
:1016B8004350030217839000FEE0C394025076E57E
:1016C8006675F00A84FF7E00900576126254E0F594
:1016D8005A755900AE59AF5A900091E012622D74B4
:1016E800648E048F05FF12621D8C5B8D5C9000EE8A
:1016F800E004C395438C068D0712622D9000EEE03E
:101708008E048F05FF12621D8C5B8D5CAE28AF299D
:10171800EF2DFDEE3CFC8C288D299000DCE0B40216
:1017280012AE2CAF2DAA5BAB5CEF2BFBEE3AFA8A1C
:101738002C8B2D80469000EEE004C39543854BF03A
:10174800A4FFAEF09000EEE08E048F05FF12621D3C
:101758008C5B8D5CAE28AF29EF2DFDEE3CFC8C2810
:101768008D299000DCE0B40212AE2CAF2DAA5BAB41
:101778005CEF2BFBEE3AFA8A2C8B2D05439000EE9A
:10178800E0C39543500375430090009BE05401600B
:101798001B90008FE0A851B80012D39552400DA2BB
:1017A8000DB3B35007E55EC394CC4002802590008A
:1017B8008DE075F003A4FFAEF0E5402FFF50010E59
:1017C80074032FFF50010EE55EBE0007D39F400350
:1017D800754401855E40E54470030218C49000EF2B
:1017E800E0C3954450030218B69000FEE0C394028B
:1017F8005076E56675F00A84FF7E009005761262E1
:1018080054E0F55A755900AE59AF5A90008EE0125F
:10181800622D74648E048F05FF12621D8C5B8D5CD3
:101828009000EFE004C395448C068D0712622D905A
:1018380000EFE08E048F05FF12621D8C5B8D5CAE9D
:1018480028AF29EF2DFDEE3CFC8C288D299000DC7B
:10185800E0B40212AE2CAF2DAA5BAB5CEF2BFBEE13
:101868003AFA8A2C8B2D80469000EFE004C3954409
:10187800854CF0A4FFAEF09000EFE08E048F05FFDA
:1018880012621D8C5B8D5CAE28AF29EF2DFDEE3CFE
:10189800FC8C288D299000DCE0B40212AE2CAF2D10
:1018A800AA5BAB5CEF2BFBEE3AFA8A2C8B2D054436
:1018B8009000EFE0C3954450037544009000F1E0B8
:1018C8002529FFAE2850010E8E288F299000A0E010
:1018D800A828B80004952950099000A0E0F52975BA
:1018E80028009000DCE0B4020D9000A0E0A82CB81D
:1018F8000006952D400280099000A0E0F52D752C7A
:1019080000229000DCE0B401028003021A15A20D47
:10191800B35003021A139000A7E0B40168AE28AFD1
:1019280029AC51AD52120003743C8E048F05FF128E
:10193800621D9000B7E0BC00109D400D9000B9E01A
:10194800A828B8000495295002D202AE28AF29ACC5
:1019580051AD52120003743C8E048F05FF12621DB4
:101968009000B7E0C3940ABC0015D39D40119000C5
:10197800B9E0C39405A828B80005D395295002807A
:1019880002C2028068AE28AF29AC51AD52120003E2
:1019980074788E048F05FF12621D9000B7E0BC00BA
:1019A800109D400D9000B9E0A828B8000495295072
:1019B80004D2028038AE28AF29AC51AD52120003D0
:1019C80074788E048F05FF12621D9000B7E0C394EF
:1019D8000ABC0015D39D40119000B9E0C39405A836
:1019E80028B80005D3952950028002C202A202B38A
:1019F8004019AE28AF299000B8E012622D74648EA9
:101A0800048F05FF12621D8C288D298002C202A254
:101A180000B34006A201B3B35009900015E4F0A347
:101A2800F08024AE28AF297400D39F74019E400C27
:101A3800900015E528F0A3E529F0800B74FF9000CD
:101A480015F8E4F0E8A3F09000BEE0D39402400C4F
:101A58009000A9E07006A20DB3B34002801AAE2828
:101A6800AF29740212622D8E288F29AE2CAF2D74E7
:101A78000212622D8E2C8F2D9000A7E0B4011AAEB1
:101A880028AF29740212622D8E288F29AE2CAF2D13
:101A9800740212622D8E2C8F2DAE28AF29745E121F
:101AA800622D740A8E048F05FF12621D8C288D2901
:101AB8009000DCE0B40217AE2CAF2D745E12622DDC
:101AC800740A8E048F05FF12621D8C2C8D2DAE2892
:101AD800AF297402BE000AD39F40067529027528F3
:101AE80000AE2CAF2D7402BE000AD39F4006752DA0
:101AF80002752C00900013E528F0A3E529F0229048
:101B08000044E090037612625FE0F541754264900C
:101B18000044E0FE9000B2E0D39E4037E55E75F0E9
:101B28000884FF7E008F37E55E75F00884ADF07C91
:101B3800008D3A753F08755903755A96E537C39471
:101B48001F5005120B99800690042BE0F537853756
:101B5800428035E55E75F00884FF7E008F37E55ECC
:101B680075F00884ADF07C008D3A753F087559030F
:101B7800755AB6E537C3941F5005120B9980069025
:101B8800044BE0F537853742229000E8E0F53C75D4
:101B98003F11755904755A00AE51AF52E53C75F0C6
:101BA8000FA4FDACF0EDD39FEC9E4021E53C8E04E4
:101BB8008F05FF12621DED75F010A4FFAEF0E55E13
:101BC80075F01184FD7C00ED2FF53D800EE55E7506
:101BD800F01184FF7E00EF24F0F53D853D37E55E8A
:101BE80075F01184AFF07E008F3A120B9985373E5D
:101BF800AE51AF529000E8E075F00FA4FDACF0EDE7
:101C0800D39FEC9E4028755904755A10853D3712AC
:101C18000B99853E38853739AE51AF52E53C8E0475
:101C28008F05FF1262488D3A853C3B120C138537AD
:101C380041754264229000E8E0F53C753F11755902
:101C480004755A00AE51AF52E53C75F00FA4FDACD7
:101C5800F0EDD39FEC9E4021E53C8E048F05FF12EA
:101C6800621DED75F010A4FFAEF0E56075F011840B
:101C7800FD7C00ED2FF53D800EE56075F01184FFC9
:101C88007E00EF24F0F53D853D37E56075F0118461
:101C9800AFF07E008F3A120B9985373EAE51AF52A6
:101CA8009000E8E075F00FA4FDACF0EDD39FEC9E3A
:101CB8004028755904755A10853D37120B99853E91
:101CC80038853739AE51AF52E53C8E048F05FF1287
:101CD80062488D3A853C3B120C1385374175426446
:101CE8009000E3E0B40479900044E0FE9000B2E094
:101CF800D39E4037E55E75F00884FF7E008F37E598
:101D08005E75F00884ADF07C008D3A753F08755912
:101D180003755A96E537C3941F5005120B99800630
:101D280090042BE0F5378537428035E55E75F0087D
:101D380084FF7E008F37E55E75F00884ADF07C0087
:101D48008D3A753F08755903755AB6E537C3941F20
:101D58005005120B99800690044BE0F53785374201
:101D68002290007CE0B4013BE56675F00A84FF7EB2
:101D7800008F37E56675F00A84ADF07C008D3A7502
:101D88003F0A755905755A12E537C3941150051263
:101D98000B998006900599E0F537E5422537C394FD
:101DA80064F54290007DE0B4013BE56775F00A8474
:101DB800FF7E008F37E56775F00A84ADF07C008DF3
:101DC8003A753F0A755905755A7EE537C39411501F
:101DD80005120B998006900605E0F537E542253790
:101DE800C39464F542E5412542F534900084E0B49B
:101DF80002109007BCE02534FE9000D8E0F4042ED1
:101E0800F5349000DBE0D394014040E56AC394E7E1
:101E1800501D74E7C3956AFE9007BEE08E00F5F08A
:101E2800E884FF7E008F37E5342537F534801CE5DC
:101E38006AC394E7FE9007BEE08E00F5F0E884FFE1
:101E48007E008F37E534C39537F534A20D4006E59B
:101E5800412464F534E534D394644009E534C394EB
:101E680064F53480037534009000B4E0C3953450B1
:101E7800069000B4E0F53422D20090006EE0A8513C
:101E8800B800049552504190006EE0A851B8000483
:101E98009552500375340F90006EE004A851B800B5
:101EA800049552500375340A90006EE02402A8513C
:101EB800B8000495525005753405C20090006EE0D4
:101EC80060067409900045F0C2387E017F009000DA
:101ED800BAE012622D9000C9E08E048F05FF1262ED
:101EE8001DE55EBC0017D39D40139000C3E0B4020B
:101EF80004D2388002C200740A900045F09000BBFA
:101F0800E0C3956650159000CDE0A851B80004953F
:101F1800525002C200740B900045F0E566C3946409
:101F2800501D900113E0600D900113E0A851B80016
:101F380006955240028008C200740B900045F0A23A
:101F48000040037534059000FCE0B401149000FDD6
:101F5800E0A851B8000495525007E55EC3955F406C
:101F68000280089000A5E0F534803A900084E0B43F
:101F78000306A228B3B34002802B9007C0E0C394A5
:101F880005A851B800049552500C9000A5E0F5340E
:101F9800740C900045F09007C0E0A851B800049573
:101FA800525002C20085346B900076E02534FE90D2
:101FB8000044E075F01E84FC7F00EE2CF53422907E
:101FC8000044E075F00584FF7E008F37900044E000
:101FD80075F00584ADF07C008D3A753F05755903A1
:101FE800755AD69000C7E01475F00584FF7E00E5A9
:101FF80037BE00039F5005120B99800BE5379004FC
:102008004C12625FE0F537E5379007BFF09007BFE5
:10201800E0FE9000B6E0C39E50089000B6E090073E
:10202800BFF022E56675F00A84FF7E0090057612FF
:102038006254E0F546E546D394644010E546C394FF
:102048006475F00F84FF7E008F468003754600900C
:102058000099E02546F546229007B0E0FEA3E0FF90
:102068007404120039E55E12622D740F8E048F0518
:10207800FF12621D9007AEECF0A3EDF090008CE02B
:10208800B40262E569C3944175F00584FF7E008F50
:1020980037E56975F00584ADF07C008D3A753F052C
:1020A800755906755A14E537C394175005120B99DC
:1020B800800690069DE0F5379007AEE0FEA3E0FFAE
:1020C800740A8E048F05FF12621DE5378C068D0792
:1020D80012622D740A8E048F05FF12621D9007AEDE
:1020E800ECF0A3EDF09007AEE0FEA3E0FF9007B49C
:1020F800E0FCA3E0FDEDD39FEC9E400F9007B4E019
:10210800F8A3E09007AEC8F0A3C8F0229006BDE09F
:10211800903419F8282873804C85527280479000B3
:10212800C9E0855EF0A4FFAEF074081200398F7222
:102138008033856072802E856672802985677280FB
:1021480024856872801F856972801A856A72801575
:102158008565728010856472800B856B728006902D
:052168000016E0F57215
:1034190002211F02212102212602213A02213F0213
:10342900214402214902214E02215302215802213D
:073439005D02216202216720
:10216D009006BEE0FE9006BFE0D39E404B9006BDAC
:10217D00E0B404189006BFE0C395725002D22990C6
:10218D0006BEE0D395724002C229802A9006BEE0B9
:10219D00C3957250099006BFE0D39572500280022C
:1021AD00D2299006BEE0D3957250099006BFE0C3C8
:1021BD0095725002C229802A9006BEE0D3957240D6
:1021CD00099006BFE0C3957240028002C2299006B5
:1021DD00BEE0C3957240099006BFE0D395724002F0
:1021ED00D229229006C1E0903440F8282873804C03
:1021FD0085527280479000C9E0855EF0A4FFAEF075
:10220D0074081200398F728033856072802E856656
:10221D007280298567728024856872801F85697236
:10222D00801A856A7280158565728010856472804A
:0C223D000B856B728006900016E0F572B5
:103440000221FB0221FD02220202221602221B029D
:10345000222002222502222A02222F0222340222C4
:073460003902223E02224363
:102249009006C2E0FE9006C3E0D39E405F9006C1AF
:10225900E0B404189006C3E0C395725002D22A90E4
:1022690006C2E0D395724002C22A803E9006C2E0BF
:10227900C3957250099006C3E0D39572500280024B
:10228900D22A9006C2E0D3957250099006C3E0C3E2
:1022990095725002C22A9006C1E0B401099000D596
:1022A900E0D3956050028002C22A802A9006C2E0DB
:1022B900D3957240099006C3E0C39572400280022B
:1022C900C22A9006C2E0C3957240099006C3E0D3C2
:1022D90095724002D22A229006C5E0903467F82808
:1022E9002873804C85527280479000C9E0855EF062
:1022F900A4FFAEF074081200398F728033856072C2
:10230900802E85667280298567728024856872802F
:102319001F856972801A856A7280158565728010B9
:10232900856472800B856B728006900016E0F572E9
:103467000222EB0222ED0222F202230602230B02C2
:10347700231002231502231A02231F0223240223E7
:073487002902232E0223336A
:102339009006C6E0FE9006C7E0D39E404B9006C5C6
:10234900E0B404189006C7E0C395725002D22B90EE
:1023590006C6E0D395724002C22B802A9006C6E0D9
:10236900C3957250099006C7E0D395725002800256
:10237900D22B9006C6E0D3957250099006C7E0C3E8
:1023890095725002C22B802A9006C6E0D3957240FE
:10239900099006C7E0C3957240028002C22B9006DD
:1023A900C6E0C3957240099006C7E0D39572400212
:1023B900D22B229006C9E090348EF8282873804CDD
:1023C90085527280479000C9E0855EF0A4FFAEF0A7
:1023D90074081200398F728033856072802E856689
:1023E9007280298567728024856872801F85697269
:1023F900801A856A7280158565728010856472807D
:0C2409000B856B728006900016E0F572E7
:10348E000223C70223C90223CE0223E20223E7024C
:10349E0023EC0223F10223F60223FB022400022472
:0734AE000502240A02240FAD
:102415009006CAE0FE9006CBE0D39E404B9006C9DD
:10242500E0B404189006CBE0C395725002D22C900C
:1024350006CAE0D395724002C22C802A9006CAE0F3
:10244500C3957250099006CBE0D395725002800275
:10245500D22C9006CAE0D3957250099006CBE0C302
:1024650095725002C22C802A9006CAE0D39572401C
:10247500099006CBE0C3957240028002C22C9006FB
:10248500CAE0C3957240099006CBE0D3957240022D
:10249500D22C229006CDE09034B5F8282873804CD4
:1024A50085527280479000C9E0855EF0A4FFAEF0CA
:1024B50074081200398F728033856072802E8566AC
:1024C5007280298567728024856872801F8569728C
:1024D500801A856A728015856572801085647280A0
:0C24E5000B856B728006900016E0F5720B
:1034B5000224A30224A50224AA0224BE0224C302D4
:1034C50024C80224CD0224D20224D70224DC0224FB
:0734D500E10224E60224EBF2
:1024F1009006CEE0FE9006CFE0D39E404B9006CDF5
:10250100E0B404189006CFE0C395725002D22D902A
:1025110006CEE0D395724002C22D802A9006CEE00D
:10252100C3957250099006CFE0D395725002800294
:10253100D22D9006CEE0D3957250099006CFE0C31C
:1025410095725002C22D802A9006CEE0D39572403A
:10255100099006CFE0C3957240028002C22D900619
:10256100CEE0C3957240099006CFE0D39572400248
:10257100D22D229006D1E09034DCF8282873804CCB
:1025810085527280479000C9E0855EF0A4FFAEF0ED
:1025910074081200398F728033856072802E8566CF
:1025A1007280298567728024856872801F856972AF
:1025B100801A856A728015856572801085647280C3
:0C25C1000B856B728006900016E0F5722E
:1034DC0002257F02258102258602259A02259F025C
:1034EC0025A40225A90225AE0225B30225B8022582
:0734FC00BD0225C20225C735
:1025CD009006D2E0FE9006D3E0D39E404B9006D10C
:1025DD00E0B404189006D3E0C395725002D22E9049
:1025ED0006D2E0D395724002C22E802A9006D2E028
:1025FD00C3957250099006D3E0D3957250028002B4
:10260D00D22E9006D2E0D3957250099006D3E0C336
:10261D0095725002C22E802A9006D2E0D395724058
:10262D00099006D3E0C3957240028002C22E900637
:10263D00D2E0C3957240099006D3E0D39572400263
:10264D00D22E229006D5E0903503F8282873804CC1
:10265D0085527280479000C9E0855EF0A4FFAEF010
:10266D0074081200398F728033856072802E8566F2
:10267D007280298567728024856872801F856972D2
:10268D00801A856A728015856572801085647280E6
:0C269D000B856B728006900016E0F57251
:1035030002265B02265D02266202267602267B02E3
:10351300268002268502268A02268F022694022608
:073523009902269E0226A377
:1026A9009006D6E0FE9006D7E0D39E404B9006D523
:1026B900E0B404189006D7E0C395725002D22F9067
:1026C90006D6E0D395724002C22F802A9006D6E042
:1026D900C3957250099006D7E0D3957250028002D3
:1026E900D22F9006D6E0D3957250099006D7E0C351
:1026F90095725002C22F802A9006D6E0D395724077
:10270900099006D7E0C3957240028002C22F900655
:10271900D6E0C3957240099006D7E0D3957240027E
:10272900D22F229006D9E090352AF8282873804CB8
:1027390085527280479000C9E0855EF0A4FFAEF033
:1027490074081200398F728033856072802E856615
:102759007280298567728024856872801F856972F5
:10276900801A856A72801585657280108564728009
:0C2779000B856B728006900016E0F57274
:10352A0002273702273902273E022752022757026B
:10353A00275C02276102276602276B02277002278F
:07354A007502277A02277FBA
:102785009006DAE0FE9006DBE0D39E404B9006D93A
:10279500E0B404189006DBE0C395725002D2309085
:1027A50006DAE0D395724002C230802A9006DAE05C
:1027B500C3957250099006DBE0D3957250028002F2
:1027C500D2309006DAE0D3957250099006DBE0C36B
:1027D50095725002C230802A9006DAE0D395724095
:1027E500099006DBE0C3957240028002C230900674
:1027F500DAE0C3957240099006DBE0D3957240029A
:10280500D230229006DDE0903551F8282873804CAF
:1028150085527280479000C9E0855EF0A4FFAEF056
:1028250074081200398F728033856072802E856638
:102835007280298567728024856872801F85697218
:10284500801A856A7280158565728010856472802C
:0C2855000B856B728006900016E0F57297
:1035510002281302281502281A02282E02283302F3
:10356100283802283D02284202284702284C022816
:073571005102285602285BFD
:102861009006DEE0FE9006DFE0D39E404B9006DD51
:10287100E0B404189006DFE0C395725002D23190A3
:1028810006DEE0D395724002C231802A9006DEE076
:10289100C3957250099006DFE0D395725002800211
:1028A100D2319006DEE0D3957250099006DFE0C385
:1028B10095725002C231802A9006DEE0D3957240B3
:1028C100099006DFE0C3957240028002C231900692
:1028D100DEE0C3957240099006DFE0D395724002B5
:1028E100D231229006E1E0903578F8282873804CA7
:1028F10085527280479000C9E0855EF0A4FFAEF07A
:1029010074081200398F728033856072802E85665B
:102911007280298567728024856872801F8569723B
:10292100801A856A7280158565728010856472804F
:0C2931000B856B728006900016E0F572BA
:103578000228EF0228F10228F602290A02290F027E
:10358800291402291902291E02292302292802299D
:073598002D02293202293740
:10293D009006E2E0FE9006E3E0D39E404B9006E168
:10294D00E0B404189006E3E0C395725002D23290C1
:10295D0006E2E0D395724002C232802A9006E2E090
:10296D00C3957250099006E3E0D395725002800230
:10297D00D2329006E2E0D3957250099006E3E0C39F
:10298D0095725002C232802A9006E2E0D3957240D1
:10299D00099006E3E0C3957240028002C2329006B0
:1029AD00E2E0C3957240099006E3E0D395724002D0
:1029BD00D23222AE2EAF2F74F5D39F74019E4008F4
:1029CD00782E126281022ADA752F01752E00AE5112
:1029DD00AF52E546BE000DD39F40099000ABE0D34A
:1029ED00954740028023754700E546C39552F57221
:1029FD009000AEE0D395454008E5452572F545803C
:102A0D00069000AEE0F54580020547900087E0D3C3
:102A1D009560401CE55EC3955F4015AE51AF52E524
:102A2D0046BE00039F50099000ACE0D3954840028C
:102A3D00806E9007C3E0A851B800049552500375FD
:102A4D004A009007C3E0A851B8000BD39552400639
:102A5D00E5529007C3F0E54A7041E552C39546F53E
:102A6D0072E572D3940540037572059000ADE0C315
:102A7D0095455007E572C3954540028009E545C36C
:102A8D009572F54580069000ADE0F5459000ADE0FE
:102A9D00D3954540069000ADE0F5457548008002A0
:102AAD000548E54A7016900087E0C39560500DE526
:102ABD00462405A851B8000695524002800F90009B
:102ACD009AE0F545754A0174789007C3F022AE2E51
:102ADD00AF2F74E9D39F74039E4008782E12628144
:102AED00022C79752F01752E00754532A233402ABF
:102AFD0075451990009AE075F002A4FFAEF0E54718
:102B0D00BE0006D39F4002D2330547754A03747841
:102B1D009007C3F0754900022C68AE51AF52E546DF
:102B2D006F4E7003022C68E546BE000DD39F400921
:102B3D009000ABE0D395474002800F754700E54A02
:102B4D00C394035003754519800DE546C39552F5A1
:102B5D0072E5472572F547900087E0D39560400EEA
:102B6D009007C3E0A851B80007D395524002800CDE
:102B7D00054990009AE0B54903754A00E54AB4034A
:102B8D0006A20DB3B34002800A0549E549B43C03E2
:102B9D00754A02E54AB402299007C3E0A851B8006E
:102BAD000ED395524009E5529007C3F07549009038
:102BBD000087E0C39560500975490074789007C38C
:102BCD00F0E54A705A900087E0D39560401CE55EB1
:102BDD00C3955F4015AE51AF52E546BE00039F5001
:102BED00099000ACE0D39548400280087548007507
:102BFD00454B8028E552C39546F572E572D3940591
:102C0D004003757205900087E0D395604008E54854
:102C1D002572F5488006E5482406F548754900E516
:102C2D004A7016900087E0C39560500DE546240567
:102C3D00A851B80006955240028003754A01E54A35
:102C4D00B40118754519054990009AE0B549067506
:102C5D004A0275490074789007C3F0E54575F00A8E
:102C6D00A4FFAEF09007B8EEF0A3EFF022E56E9062
:102C7D00359FF828287390007FE07003022E28906E
:102C8D0000B5E0B401028003022D78900042E0B55A
:102C9D005D028003022D757E017F00E5BE12622D5F
:102CAD00E5BD2FFF50010E8E598F5A741012622DF3
:102CBD0090006DE08E048F05FF12621D9007C4EC2D
:102CCD00F0A3EDF0E56A60089000DBE064026002BD
:102CDD0080269000DDE0B4011F9007C4E0FEA3E064
:102CED00FF74E712622DE56A8E048F05FF12621DD7
:102CFD009007C4ECF0A3EDF090007FE0B4022790B4
:102D0D0007C6E0FEA3E0FF9007C4E0FCA3E0FDEFE3
:102D1D002DFDEE3CFC74018C068D071200399007D9
:102D2D00C4EEF0A3EFF09007C4E0FEA3E0FF900720
:102D3D00C6E0FCA3E0FDEDD39FEC9E4004D23680AF
:102D4D0002B2369007C4E0F8A3E09007C6C8F0A31E
:102D5D00C8F09000B1E064016006A236B3B3400242
:102D6D0080069007C5E0F55E022E26D2367E017FE5
:102D7D0000E5BE12622DE5BD2FFF50010E8E598F5D
:102D8D005A741012622D90006DE08E048F05FF12A3
:102D9D00621D9007C4ECF0A3EDF0E56A60089000A9
:102DAD00DBE06402600280269000DDE0B4011F903C
:102DBD0007C4E0FEA3E0FF74E712622DE56A8E04FE
:102DCD008F05FF12621D9007C4ECF0A3EDF090008B
:102DDD007FE0B402279007C6E0FEA3E0FF9007C492
:102DED00E0FCA3E0FDEF2DFDEE3CFC74018C068DA7
:102DFD00071200399007C4EEF0A3EFF09007C4E07E
:102E0D00F8A3E09007C6C8F0A3C8F09000B1E06445
:102E1D000160069007C5E0F55E8003755E009000C9
:102E2D007BE07006756E01022C7A75BB180233F3C8
:102E3D0090007BE07003022FC97E017F00E5BE127A
:102E4D00622DE5BD2FFF50010E8E598F5A9000C196
:102E5D00E0B4010F7E0F7FFFAC59AD5A1262798E2F
:102E6D00598F5A9000E6E0B40245AE59AF5A900022
:102E7D001FE0FCA3E0FDEDD39FEC9E400A90001FE8
:102E8D00E559F0A3E55AF0AE59AF5A900021E0FC98
:102E9D00A3E0FDEFD39DEE9C400A900021E559F093
:102EAD00A3E55AF0AE59AF5A74041200398F6090F1
:102EBD0000E6E0704CAE59AF5A90001FE0FCA3E065
:102ECD00FDEFD39DEE9C40091262798E598F5A8089
:102EDD0006755A00755900AE59AF5A741012622D0D
:102EED0090006AE08E048F05FF12621D8C598D5A79
:102EFD0074FFBC0009D39D4005855A608003756041
:102F0D00FE9000B1E0B401028003022FC7A20DB301
:102F1D00B3500E900085E0A851B80005D3955250DE
:102F2D0003022FBC900086E075F019A4FFAEF0905F
:102F3D0000C9E08E048F05FF12621D9000C2E0856E
:102F4D0060F0A4FFAEF074648D028C038E048F05C7
:102F5D00FF12621DEA2DFDEB3CFC8C598D5AE56A82
:102F6D00600F9000DBE0B402089000DDE0640160CA
:102F7D00028017AE59AF5A74E712622DE56A8E04BE
:102F8D008F05FF12621D8C598D5AAE59AF5A90079D
:102F9D00C4E0FCA3E0FDEDD39FEC9E4005855A5E99
:102FAD00800BA236B340069007C5E0F55E800BA2FC
:102FBD0036B340069007C5E0F55E8003756000905E
:102FCD00007EE07006756E02022C7A75BB19023315
:102FDD00F390007EE0700302307EE55DD3955040A6
:102FED000302307C90001DE0FEA3E0FFE564126259
:102FFD007190001DEEF0A3EFF07E017F00E5BE1293
:10300D00622DE5BD2FFF50010E8E598F5A9000EBAA
:10301D00E07013740A12622D74518E048F05FF1225
:10302D00621D8D648019AE59AF5A740A12622D8FCC
:10303D00048E057E017F95CDCCCD12611B8F64E58D
:10304D0064D39464400375646490001DE0FEA3E0B6
:10305D00FFE5642FFF50010E90001DEEF0A3EFF081
:10306D00900082E0048E048F05FF12621D8D648036
:10307D00037564329000CEE07006756E03022C7AF3
:10308D0075BB130233F39000CEE0604A7E017F00E2
:10309D00E5BE12622DE5BD2FFF50010E8E598F5AE0
:1030AD0074041200398F659000D0E08565F0A4FDA1
:1030BD00ACF07464FF12621D8D659000CFE08565E4
:1030CD00F0A4FFAEF074FF8E048F05FF12621DEDAC
:1030DD00900069F0800375650090007CE0700675C6
:1030ED006E04022C7A75BB170233F390007CE0B4AA
:1030FD000102800302318C7E017F00E5BE12622D3C
:10310D00E5BD2FFF50010E8E598F5A9007C8E06014
:10311D00199007C8E014905CAD12008CE493FC7418
:10312D000193FDEDC39FEC9E400280069007C8E021
:10313D0014F09007C8E0C394B3501DAE59AF5A9028
:10314D0007C8E004905CAD12008CE493FC7401930D
:10315D00FDEFC39DEE9C400280069007C8E004F091
:10316D009007C8E0FE9000A2E08E0088F0A4FFAEAC
:10317D00F074648E048F05FF12621D8D66800375D9
:10318D00660090007DE07006756E05022C7A75BBA9
:10319D00160233F390007DE0B40102800302323554
:1031AD007E017F00E5BE12622DE5BD2FFF50010EA1
:1031BD008E598F5A9007C9E060199007C9E0149095
:1031CD005E1712008CE493FC740193FDEDC39FEC2C
:1031DD009E400280069007C9E014F09007C9E0C335
:1031ED0094B3501DAE59AF5A9007C9E004905E17C5
:1031FD0012008CE493FC740193FDEFC39DEE9C4093
:10320D000280069007C9E004F09007C9E0FE900027
:10321D00A8E08E0088F0A4FFAEF074648E048F05D4
:10322D00FF12621D8D67800375670075BB1F02332A
:10323D00F37E017F00E5BE12622DE5BD2FFF50012B
:10324D000E8E598F5A740912622D74E68E048F05F5
:10325D00FF12621D8D69900084E07006756E070285
:10326D002C7A75BB150233F3900084E070030233A2
:10327D008F7E017F00E5BE12622DE5BD2FFF50014F
:10328D000E8E598F5A74041200398F68900084E0A5
:10329D00B401159000D8E08568F0A4FFAEF0740776
:1032AD00120039EF9007BDF0900084E0B402159044
:1032BD0000D8E08568F0A4FFAEF07407120039EF76
:1032CD009007BCF0900084E0B40302800302338DBC
:1032DD009000C5E070389000D8E0601CE568C3949C
:1032ED00195002D228E568D394644002C228900098
:1032FD00A4E09007C0F08014E568C394195002D281
:10330D0037E568D394324002C237C22880639000FB
:10331D00A4E070349000D8E08568F0A4FFAEF0749E
:10332D00FF8E048F05FF12621DED9007C0F0AE51A8
:10333D00AF52741EBE0006D39F4002D228E560D363
:10334D0094E54002C2288029E568C3940A500DAE69
:10335D0051AF52741EBE0004D39F50028002D2287A
:10336D00E560D394E54002C2289000A4E09007C028
:10337D00F09007C0E0C39405500674059007C0F0A7
:10338D0080037568009000DBE07006756E08022CF6
:10339D007A75BB1480509000DBE060397E017F00B0
:1033AD00E5BE12622DE5BD2FFF50010E8E598F5ACD
:1033BD00EFD39421EE940E4005756AFF8015AE593A
:1033CD00AF5A741012622D74E38E048F05FF1262D2
:1033DD001D8D6A8003756A0090007FE0600575BBE6
:0633ED001A800375BB18F5
:10359F00022C83022E3D022FDE0230930230F802FE
:0B35AF0031A102323E0232750233A34C
:0533F300056ED2EC2282
:09625F002582F58250020583221C
:0F008C0025E050020583258250020583F582226C
:1061FC00EF2F500205832582F582E5833E2EF58331
:01620C00226F
:10627100CFC39FFF50011E22C3EF9DFFEE9CFE2264
:086281000806B600021806220F
:0D623B00A3E004F07006120049E004F02218
:0E003900048007C3CE13CECF13CFD5E0F6223E
:10611B00BC000FBE0008ED8FF084FFADF022E4FE53
:10612B00FF22BE000DEF60FE54F0606F20E703020C
:10613B0061D1EAC0E0EBC0E078017A0075F001EEC6
:10614B0020E710EF25E0FFEE33FE0AC5F023C5F084
:10615B0030E7F0EA5407F9096A7A007B006001081E
:10616B00C3EC9E40167004ED9F4010ED9FFDEC9E1E
:10617B00FCE5F0CA4ACA03F5F08005E5F003F5F03B
:10618B00C3EE13FEEF13FFD9D77908CACBCAD8D009
:10619B00EAFEEBFFD0E0FBD0E0FA22EC8FF084FCC0
:1061AB00ED54F045F0C48FF084FEEDC454F045F08F
:1061BB00C48FF084FDEEC4FE54F02DFFEE540F3C63
:1061CB00FEADF07C0022790078008FF0EC7E082089
:1061DB00E70DC3CD33CD33C933C9C833C8DEF08423
:1061EB0049F9E5F08FF0BE00E6FD7C00E9FFE8FE23
:0161FB002281
:0E622D00F88FF0A4FFE5F0CE88F0A42EFE223C
:10000300EF8DF0A4F9A8F0EF8CF0A428F8EE8DF0B2
:06001300A428FEE9FF2213
:10620D00600D782B026217007830D8FED5E0F822A9
:10621D00EEC0E07E0012611BEFFDEEFCD0E0FE2231
:0C624800EEC0E07E0012611BD0E0FE22E0
:03001B0002001EC2
:0300530002005652
:03009B00020071EF
:0300000002626831
:0962680075817475D0000240023A
:0B625400E5822FF582E5833EF58322F2
:0A0049000582D5820215831582227C
:10001E00C0E0C0F0C083C082C0D075D000123F3C9B
:0B002E00D0D0D082D083D0F0D0E032E0
:10005600C0E0C0F0C083C082C0D075D000123F3F60
:10006600D0D0D082D083D0F0D0E032C0E0C0F0C093
:1000760083C082C0D075D000123FC4D0D0D082D009
:0600860083D0F0D0E0324F
:00000001FF
